:020000020000FC
:0200000002C03C
:100004000FC000E107BB0FE008BB00E20BBF0FE02D
:1000140005BB00E305BF00E808B978948895FECFD6
:1000240016B31F701F3011F004D0FACF0FE008BBD5
:100034001895512F529510951F70512B09E4000FFC
:10004400402F102702951027012F1695169501278A
:10005400102F169501270170402B01D0089525E03B
:100064007A0130E1F7FE13D0F7FC17D00CD0EE0C78
:10007400FF1C3A95B9F707D006D005D004D02A95CD
:1000840009F0EECF089500E50A95F1F70895C49AB2
:1000940008E20A95F1F7C4980895C49A00EA0A950B
:0600A400F1F7C498089575
:00000001FF
